:1018000026C044C05DC042C041C040C03FC03EC0D1
:101810003DC03CC03BC03AC039C038C037C00902E7
:1018200019000101008032090400000100000000DD
:101830000705810308006412011001FF000008D0B1
:101840001653070A010000000104030904001124D3
:101850001FBECFE5D2E0DEBFCDBF00EB0F9307E0A8
:101860000F9310E0A0E6B0E0EEEEFFE102C00590BD
:101870000D92A636B107D9F720E0A6E6B0E001C088
:101880001D92A73AB207E1F70CD2AFC3B9CFA82F88
:10189000B92F80E090E041E050EA609530E009C067
:1018A0002D9182279795879510F084279527305E94
:1018B000C8F36F5FA8F30895EADF8D939D930895B1
:1018C000CF93CFB7CF93C0915F02C03B21F4C091BB
:1018D0005E02C73021F0CF91CFBFCF9190CFCC2700
:1018E000C395B39BE9F7B39B0BC0B39B09C0B39BF4
:1018F00007C0B39B05C0B39B03C0B39B01C0D5C059
:101900000F92DF93C0918A00DD27CF56DF4F012E63
:10191000B39B03C0DF910F90E6CF2F930F931F93DC
:101920004F932FEF4F6F06B303FB20F95F933F9365
:1019300050E03BE065C016B30126502953FDC89521
:1019400056B3012703FB25F92F7306B3B1F05027D7
:10195000102713FB26F906B22230F0F000C016B3B0
:10196000012703FB27F90126502906B22430E8F5A8
:101970004F77206816B30000F6CF50274F7D2062C6
:1019800006B2102F000000C006B300265029102711
:1019900013FB26F906B2E2CF4F7B06B3206400C0EA
:1019A000DACF01265029187106B269F14E7F216005
:1019B000012F16B328C0002650294D7F06B22260A1
:1019C000102F29C0012650294B7F06B22460012F19
:1019D0002DC016B301265029477F2860000006B2AB
:1019E0002EC04F7E06B3206130C0422706B3499314
:1019F00000265029102706B24FEF13FB20F9297F4C
:101A000016B379F2187159F10126502906B201274F
:101A100003FB21F9237F06B371F2002650293150D0
:101A2000D0F006B2102713FB22F9277E16B351F22D
:101A300001265029012703FB06B223F92F7C49F226
:101A4000000006B3102713FB24F90026502906B224
:101A50002F7939F270CF10E21ABF002719C03B501E
:101A60003195C31BD04010E21ABF0881033C09F135
:101A70000B34F9F0209188001981110F1213EDCF6A
:101A80004A81441F093651F10D3211F0013E29F708
:101A900000938F003F915F914F911F910F912F9174
:101AA000DF910F90CAB7C5FD1BCFCF91CFBFCF91AC
:101AB000189520918F00222369F310918D00112336
:101AC00079F534307AF130938D00209389001091AC
:101AD0008A003BE0311B30938A0024C000918D00C6
:101AE0000130F4F40AE54F7049F43091600034FDA0
:101AF0001AC000936000C1E7D0E019C030917C00AB
:101B000034FD11C000937C00CDE7D0E010C0052764
:101B100010E000C021C0052710E0C89508BB14C024
:101B20003AE501C032ED032EC0E0D0E032E017B359
:101B30001861C39A08B317BB58E120E84FEF20FFA4
:101B4000052708BB279517951C3F28F7000045522D
:101B5000B0F720FF0527279508BB17951C3FB8F65F
:101B600029913A9561F7077E10918E00110F08BBFD
:101B7000C250D04011F01093880010E21ABF0860E4
:101B800017B3177E402F477E54E05A95F1F708BBF4
:101B900017BB48BB7FCFF8942FEFB0E8A0E44AE032
:101BA000B1BF000081EE9CE0B399FECFB39BFECFA6
:101BB0000197B399FDCF97FF03C0BA1B819501C070
:101BC000BA0FA69529F4281710F031B7282FA1E0F5
:101BD000415031F731BF0000789408958FB7F894E1
:101BE000E0916900F0916A00329795E09093570078
:101BF000E8958FBF08952091690030916A00211502
:101C0000310539F490936C0080936B008FEF9BEC5F
:101C100027C02430310539F490936E0080936D0015
:101C20008FEF9BEC23C02C3F47E1340739F48091C0
:101C30006B0090916C008E5F9B4F18C02E3F47E168
:101C4000340739F480916D0090916E008D5F9B4F49
:101C50000DC02A3F47E1340719F481B790E006C070
:101C6000232B21F421E120935700E8952FB7F89416
:101C7000E0916900F0916A0031E00C013093570067
:101C8000E89511242FBF3296F0936A00E093690023
:101C900008958FEF9FEFAFDF809169008F73C9F7D1
:101CA0009DCF2EE088E190E00FB6F894A89581BD15
:101CB0000FBE21BDE1E0F0E0E491EF3F09F4E9DF80
:101CC00010926A0010926900BB9A88EB9BE0ECE9E5
:101CD000F1E03197F1F70197D1F7BB98AC9A8BB748
:101CE00080628BBF8BE480937D008AE580937C00CB
:101CF000789400918D00035007FDC7C080918A0041
:101D0000CCE0D0E0C81BD109CF56DF4F80918900CD
:101D10008D3209F09BC0083009F0B5C083EC809388
:101D200071008AE58093600010926F002881922FE5
:101D300090768981992329F11092670010926600AC
:101D4000811108C082E690E090938C0080938B0014
:101D500014E072C0813051F48C819D8190936A00AF
:101D60008093690027FD63C01FEF62C090916800F7
:101D7000823011F4916001C094609093680010E08B
:101D80005BC09A8110927A00811106C010927B008C
:101D90008AE790E012E046C0853019F490938E00F7
:101DA0003EC0863031F58B81813041F487E398E184
:101DB00090938C0080938B0012E117C0823041F425
:101DC0008EE198E190938C0080938B0019E10DC017
:101DD000833051F4911108C089E498E190938C000C
:101DE00080938B0014E001C010E080E480936F00CA
:101DF00023C0883069F0893019F4909390000FC0A7
:101E00008A3049F08B3059F48BE480937D0007C011
:101E100080E990E002C08AE790E011E003C08AE721
:101E200090E010E090938C0080938B0005C01E81A1
:101E300080E880936F0007C08F81811104C08E817C
:101E4000811708F4182F109361001DC080916F0056
:101E500087FF19C08091690090916A0081159841AF
:101E600028F0809169008F7339F00DC089919991A4
:101E7000C2DE025079F7F5CF8091680082608093CE
:101E800068001092610010928D008091600084FFC4
:101E900043C0809161008F3F09F43EC0082F893014
:101EA00008F008E0801B809361008091710098E841
:101EB000892780937100002319F1E0918B00F09144
:101EC0008C0080916F0086FF0BC0A2E7B0E0849188
:101ED0008D93319682E790E0800F8A13F8CF0CC083
:101EE000CF01A2E7B0E0FC012191CF012D9322E7C1
:101EF00030E0200F2A13F7CFF0938C00E0938B0093
:101F0000602F82E790E0D8DC0C5F0C3019F08FEF87
:101F1000809361000093600084E196B3987131F47E
:101F20008150D9F710928E001092880001E0811143
:101F300000E080917000801739F0011103C0109209
:101F4000670029DE00937000A8958CE991E0019765
:101F5000F1F78091680080FF11C0F894E0E0F8E1AB
:101F6000E054F10983E080935700E8953097C1F77A
:101F700010926A00109269008CDE789400916800DB
:101F800001FF05C08AE390E20197F1F727DE02FF27
:101F900018C082E291EA0197F1F7F894BB9A88E1C0
:101FA0000FB6F89481BD11BC0FBE1BBE15BA1092BE
:101FB0005F02EAEFF7E1E4918E2F81508E3F88F0C7
:101FC00012C010926800809166009091670001969F
:101FD000909367008093660080369A4E08F489CE0D
:0E1FE000D8CFE1BF00000ACC27CFF894FFCF86
:061FEE005AFF17FA40083B
:0400000300001800E1
:00000001FF
